:020000040802F0
:1040000000C00020115A0208995B0208255D0208D1
:10401000395D02083D5D0208415D020800000000B4
:104020000000000000000000000000000000000090
:104030000000000000000000000000000000000080
:104040000000000000000000000000000000000070
:104050000000000000000000000000000000000060
:104060000000000000000000000000000000000050
:104070000000000000000000000000000000000040
:10408000000000000000000000000000455D020884
:10409000495D020800000000000000000000000070
:1040A0000000000000000000000000000000000010
:1040B000000000004D5D020800000000000000004C
:1040C00000000000000000000000000000000000F0
:1040D00000000000000000000000000000000000E0
:1040E00000000000000000000000000000000000D0
:1040F00000000000000000000000000000000000C0
:1041000000000000000000000000000000000000AF
:10411000000000000000000000000000000000009F
:10412000000000000000000000000000000000008F
:104130002DE9F04385B0E0F773F84FF4A056002066
:10414000E0F768F8C4F20106E0F76AF84FF0C044FF
:104150004FF48051EF207161208000BF00BF00BF8D
:1041600000BF00BF00BF00BF00BF00BF00BF316184
:1041700023884FF0C0421588B2F800C01488B2F806
:1041800000905FFA8CF75FFA89F848EA056646EA1C
:104190000741200648F2641441EA1045C0F60204C3
:1041A000B4214FF6FF72002314208DE8300000F098
:1041B0007FFA48F27813C0F602034FF2E0720093E0
:1041C000C1F6FF721588284C00271420A0214FF655
:1041D000FF72002348F294190195C0F6020900F01D
:1041E00067FA3D46BC4604F10408CFF20F07D4F845
:1041F00004E0261DBE4505F1010506F1040408EBA7
:104200008C0C4FF078014FF6FF724FF000034FF027
:10421000140003D08DE8005200F04AFA766808EBEB
:10422000850EBE424FF014004FF078014FF6FF723A
:104230004FF0000304D08DE80042029600F038FAF7
:104240000135B5F5005FAC46D1D148F2A414C0F6F3
:104250000204142078214FF6FF7200238DE810012C
:1042600000F026FAFEE700BFFC3F0608CB790122EA
:104270009842F0B4CF6831D303FB02F2B0FBF2F402
:104280009C42F9D2A2B100252E1C18BF0126002C99
:10429000C8BF46F0010602FB1400B2FBF3F25EB9A0
:1042A0001AB13546B0FBF2F4EEE7303407F8014BB3
:1042B00000203870F0BC70473023092C04DD0B7AE5
:1042C000002B0CBF572337231C1907F8014B002A7A
:1042D000EED00135CB79B0FBF2F4D5E70446D2E756
:1042E0002DE9F843D36817461A7805460E463C6810
:1042F000A2B1002C12DD13F8010F013C04F0010102
:1043000060B15CB109B104E044B113F8011F013C94
:1043100021B113F8012F013C002AF5D1797901B1BF
:10432000013CBB792BB1FB79102B63D0082B08BF64
:10433000013C387920BB631E002CD8BF1C461FDD12
:1043400020214FF00108284603EA0809B047A0459C
:1043500013D0B9F1000F06D0202128464FF00208F3
:10436000B047A04509D020212846B04708F10208EF
:1043700020212846B047A045F5D179794FF0FF3488
:10438000002934D1B97921B1FB79102B34D0082B15
:104390003DD03B7903B3002C1EDD04F1FF32302108
:1043A0004FF00108284602EA0809B047A04513D09B
:1043B000B9F1000F06D0302128464FF00208B0476F
:1043C000A04509D030212846B04708F10208302125
:1043D0002846B047A045F5D1FC68217829B1284688
:1043E000B04714F8011F0029F9D1BDE8F883284629
:1043F000B047C7E7023C9CE728463021B0473A7AED
:104400002846002A0CBF78215821B047C1E728462A
:104410003021B047BDE700BF436882680133934253
:104420003DBF0268436002F8011B436038BF026071
:10443000704700BF2DE9F04389B00027984605ABCF
:1044400006460D4614460493B9462178002944D007
:10445000013425293CD10023CDF804908DF8097052
:10446000184614F8011B002937D0232963D03029BE
:104470005FD0A1F130025FFA82FC8DF80830002392
:10448000BCF1090F8DF80A0012D8D0B2A1F1610C6D
:1044900009285FFA8CFC23D9A1F14102BCF1050F78
:1044A000D2B298BFA1F1570223D80A2A18DD01938E
:1044B0006C2908BF14F8011B69294FD03DD8632926
:1044C0006BD048D858291DD0BFD831B12529BCD1CF
:1044D0003046A84721780029BAD109B0BDE8F08359
:1044E00014F8011B03EB830002EB4003A1F130023F
:1044F000CBE7052ADBD8A1F13702D6E7752938D0FA
:104500007829A2D1A1F15801484240EB010E1023B5
:10451000D8F8000001A98DF80B308DF80CE008F1F7
:104520000408FFF7A3FE3046294601AAFFF7D8FE8C
:104530008BE7012395E7012093E7732922D0DDD88B
:104540006F2982D10822D8F8000001A98DF80B202C
:1045500008F10408E5E764297FF477AFD8F8000094
:104560000A2100288DF80B1008F104081CDB01A9B2
:10457000D7E70A23D8F8000001A98DF80B3008F11D
:104580000408CEE7D8F800303046294601AA08F1E1
:1045900004080493FFF7A4FE57E798F8001030468C
:1045A00008F10408A84750E72D2240428DF8092061
:1045B00001A9B6E710B584B0039144F21941019006
:1045C000002401A8C0F602010294FFF733FF019B0B
:1045D0001C70029804B010BD0CB410B582B004ACCD
:1045E00054F8042B23460194FFF7E4FF02B0BDE822
:1045F000104002B0704700BFF8B59CF80230644626
:10460000154613B1024608461146C1F30F21C0F307
:104610000F20DFF7FBFDDFF727FE45F25657C5F504
:1046200080725500C5F2555787FB051600F4784394
:10463000C6EBE5756E4200F4FC614FEA2322CF1011
:10464000238802FB06F2C00007FB06F75FFA80FC36
:1046500003F4784105F5807503F4FC640CFB06F661
:10466000091201FB0521E210D80002FB0572C4B259
:1046700004FB056C01F1FF0331EA210128BF194653
:1046800002F1FF0032EA220228BF0246CC12931246
:10469000E2020CF1FF0442EA43113CEA2C0C28BF71
:1046A000A44641EAEC2080B2BDE8F840DFF7B0BD97
:1046B0002DE9F04385B00DF1300E5EF804CB43F2E6
:1046C0000414C2F2000406460F4615469846624698
:1046D000734637212046CDF80CE0FFF76BFF3946D3
:1046E00081462A46304643460094DFF7ADFD4846F2
:1046F00005B0BDE8F08300BF08B42DE9F04F8AB0E3
:1047000013AD55F8043B05900395924600F1100255
:104710000398894648F2082147F29827C0F602011B
:10472000041D139307924FF000080491C2F2000792
:1047300006944FF6487B0020049C494602460346F7
:104740000094FFF7B5FF139D494652460023059894
:104750000095DFF779FD139803F0D4FC039C0699CC
:10476000246809912546E4B1079E002506EBC006A2
:10477000C8EB050CDCF1000040EB0C035246B0B274
:1047800049460094DFF760FD204603F0BBFC099B1F
:1047900002301A1D09921C6806EBC0060135002C78
:1047A000E6D164213980B7F800E01FFA8EF4002CBE
:1047B000F9D10420DFF74EFD80F47E4080F4A4742C
:1047C00048F2480204EA0203002BF2D00420DFF78B
:1047D00041FD5845FAD164213980B7F800C01FFA6D
:1047E0008CF3002BF9D1B8F1000FD4BF00230123C3
:1047F00013EAD40318BF08F1FF389CD1220405D571
:10480000013DA845B8BF08F1010894DB630692D5C5
:1048100040460AB0BDE8F04F01B070472DE9F04FB7
:1048200083B0BDF830700D461E464FF0874100231F
:1048300014468DF80630ADF8047003F051FA03F019
:1048400015FC4FF087418246204603F049FA03F0F9
:104850000DFC4FF087410446284603F041FA03F06F
:1048600005FC4FF087410546304603F039FA03F066
:10487000FDFBCAEB0403C5EB000883EAE371A1EB7F
:10488000E37188EAE872A2EBE87291420646274695
:10489000504609DA9946012143463446AA468DF826
:1048A0000610C8463E460546544505DAAB46504616
:1048B0003546A2465E4604460AF1800222F0FF0712
:1048C0004FEA082191FBF3F8CAEB070308FB03FA50
:1048D0000AF1FF0E3AEA2A0A28BFF24605EB2A2B14
:1048E000D0B25FFA8BF5C0F58079C5F5807101FB18
:1048F00009F32BF0FF0A1A1238460DF1040C514649
:10490000FFF77AFE05FB09F204F1800525F0FF09A7
:10491000384612120DF1040C0AF58071FFF76CFE97
:10492000C4EB090008FB00F101F1FF0331EA2101AA
:1049300028BF194606EB212C5FFA8CF4C4F580766B
:10494000EDB206FB05F204FB05F42CF0FF06121293
:104950000DF1040C48463146FFF74EFE0137220A9E
:104960000DF1040C484606F58071FFF745FE4F45F2
:104970005ADA0BEB080525F0FF065FFA85FAF843D3
:1049800000EB09043146CAF580720DF1040C38467B
:10499000FFF732FEC4F3002B0DF1040C07F5807411
:1049A000384606F580715246FFF726FE4C454544D1
:1049B0003ADABBF1000F09D025F0FF07EEB220462E
:1049C0003946C6F580720DF1040C1EE025F0FF0794
:1049D000EEB220463946C6F5807245440DF1040C0E
:1049E000FFF70AFE204607F5807132460DF1040CF0
:1049F00004F5807425F0FF07EEB2FFF7FDFD3946A0
:104A0000C6F580720DF1040C2046FFF7F5FD204637
:104A10000DF1040C07F58071324604F58074FFF740
:104A2000EBFD4C454544D1DB03B0BDE8F08F00BF42
:104A300088422DE9F04105460C461E462CDC97B213
:104A40003946221A80B2C2F340080235DFF7DEFB96
:104A50003046DFF7DDFBAC4220DBB8F1000F09D0B8
:104A6000A8B23946DFF7D2FB02353046DFF7D0FB7C
:104A7000AC4215DB3946A8B2DFF7C8FB0235304639
:104A8000DFF7C6FBA8B23946DFF7C0FB0235304678
:104A9000DFF7BEFBAC42EDDABDE8F081BDE8F081A6
:104AA000BDE8F08191422DE9F0410C4615461E46C5
:104AB0002CDC87B2121B89B23846C2F3400802349C
:104AC000DFF7A4FB3046DFF7A3FBA54220DBB8F1FC
:104AD000000F09D0A1B23846DFF798FB0234304608
:104AE000DFF796FBA54215DBA1B23846DFF78EFB58
:104AF00002343046DFF78CFBA1B23846DFF786FB85
:104B000002343046DFF784FBA542EDDABDE8F081E0
:104B1000BDE8F081BDE8F081F8B50278002A60D0E8
:104B200043F20417C2F20007002307F1380E07F121
:104B30003F05202109E0204610F8016B07EB030C2C
:104B40008CF838606278013342B32E2A18BF0446CD
:104B5000F1D1441C072BEEDC5E1E0EEB0602D343A4
:104B6000E818531CAB42517000F001000AD018B194
:104B700003F8011FAB4205D0581C59700233AB42F9
:104B80004170F9D12046082310F8016B07EB030CA4
:104B90008CF8386062780133002AD6D10A2B12DCF7
:104BA00011485A1C20210A2AC15403F001030ADCCF
:104BB0001BB1815401320A2A05DC531C8154023294
:104BC0000A2AC154F9DD0948A0F10C0100F516725A
:104BD00000F51873DFF75AFBD0F1010038BF002051
:104BE000F8BD13460048DCE73C3100204831002086
:104BF000F8B50278002A6BD043F20414C2F2000424
:104C0000002304F1380E04F13F06202109E0284674
:104C100010F8017B04EB030C8CF838706A780133D0
:104C200042B32E2A18BF0546F1D1451C072BEEDCF6
:104C30005F1E0EEB0702D343F018531CB3425170B2
:104C400000F001000AD018B103F8011FB34205D0EB
:104C5000581C59700233B3424170F9D128460823D9
:104C600010F8017B04EB030C8CF838706A78013380
:104C7000002AD6D10A2B12DC18495A1C20200A2AF5
:104C8000C85403F001030ADC1BB1885401320A2A1C
:104C900005DC531C885402320A2AC854F9DD104836
:104CA000A0F10C0100F5167200F51873DFF7ECFAAD
:104CB0000021C1EB000EDEF1000242EB0E0084F891
:104CC000A802C4F8AC12C4F8B012C4F8B412F8BD0B
:104CD00002491346A1F13804CFE700BF3C31002060
:104CE0004831002038B543F20414C2F2000494F8AD
:104CF000A8327BB1D4F8B032D4F8AC22E118013339
:104D00000132B3F5007F81F84400C4F8B032C4F832
:104D1000AC2200D238BDD4F8B4020025421C04F500
:104D2000277104F14400C4F8B052C4F8B422DFF78C
:104D3000B1FA0028EED084F8A85238BD0846FFF733
:104D4000D1BF00BF38B543F20414C2F2000494F896
:104D5000A80218B917E02020FFF7C4FFD4F8B0323A
:104D6000002BF8D10848D4F8B4220025510200F5F0
:104D7000187300F5167284F8A852DFF78DFA411BFC
:104D8000484240EB010038BD483100200FB470B5F7
:104D900082B006AE56F8042B43F2041444F63D519B
:104DA000C2F200040020C0F602013346D4F8AC522F
:104DB0000196FFF73FFBD4F8AC02401B02B0BDE800
:104DC000704004B0704700BF70B50646002409E08B
:104DD0000D48FFF701FC0C48FFF79EFE90B1B4F5BB
:104DE0007A7F0FD023460D2132460748FFF7F4FBA8
:104DF0000548FFF791FE651C0D21023432462B4613
:104E00000028E5D1004870BDBC3300202DE9F00F2B
:104E1000C10000F4FC65ED10C9B200F47840041242
:104E2000A5F1FC0BA1F1F8000028B8BF4042BBF18E
:104E3000000FB8BFCBF1000BA4F1F80700EB0B0398
:104E4000002FB8BF7F4286B04A190193A218DB1920
:104E50009A4200F3BB8013460022A5F18006A1F11F
:104E6000800CBCF1000FB8BFCCF1000C86EAE67AEA
:104E7000AAEBE67AA4F18006002EB8BF76420CEBCE
:104E80000A0808EB06094B45C4BF4B46022285EAD7
:104E9000E579A9EBE57948440390CDF808A0DDF861
:104EA0000CA084EAE470A0EBE4700AEB0008434530
:104EB000C4BF4346032281EAE178A8EBE1780BEB1B
:104EC000080ACDF810A082445345C8BF5346CDF818
:104ED00014A009EB080ACDF814A0BA44C8BF0422F4
:104EE0005345C8BF5346CDF800A0DDF804A0C8BFA5
:104EF000052282445345C8BF5346CDF800A0DDF8D3
:104F000010A0C8BF0622BA445345C8BF5346CDF8C7
:104F100010A0DDF80CA0C8BF07225744BB42C8BF91
:104F20003B460CEB09070744C8BF0822BB42C8BF79
:104F30003B46029FC8BF092207EB080900EB09089E
:104F40004345C8BF4346DDF81480C8BF0A2206EBBC
:104F500008094B450BEB0C00C8BF4B4606EB00099C
:104F6000C8BF0B224B45C8BF4B46DDF80490C8BFF5
:104F70000C224E44B342C8BF3346A1F1600CC8BFF7
:104F80000D22BC3D002DB8BF6D42BCF1000FB8BF73
:104F9000CCF1000C603C002CB8BF64420CEB050067
:104FA00000EB040C6345A1F1B801C4BF63460E22B7
:104FB0000029B8BF4942481900EB040C9C45ACBF1E
:104FC00010460F2006B0BDE8F00F7047012244E7FD
:104FD000F8B5FFF70DFE864C04F136066078651CC7
:104FE000FFF780FE02346878FFF77CFEB442F5D10B
:104FF0000020FFF777FE0020FFF774FE0020FFF788
:1050000071FE0020FFF76EFEF820FFF76BFEFC201C
:10501000FFF768FEF820FFF765FE0020FFF762FE4D
:105020008020FFF75FFE8020FFF75CFE8020FFF707
:1050300059FE0020FFF756FE0020FFF753FE002028
:10504000FFF750FEF820FFF74DFE0020FFF74AFE65
:105050000020FFF747FEFC20FFF744FE0020FFF78B
:1050600041FE0020FFF73EFEF820FFF73BFE002048
:10507000FFF738FE0020FFF735FE0020FFF732FE75
:105080000020FFF72FFEFC20FFF72CFEF820FFF793
:1050900029FE0020FFF726FEF820FFF723FEFC2064
:1050A000FFF720FE0020FFF71DFE0020FFF71AFE8D
:1050B000F820FFF717FE0020FFF714FEF820FFF797
:1050C00011FE0020FFF70EFE0020FFF70BFE002070
:1050D000FFF708FE8020FFF705FE0020FFF702FE25
:1050E0000020FFF7FFFD8020FFF7FCFD0020FFF709
:1050F000F9FD0020FFF7F6FD8020FFF7F3FD00200B
:10510000FFF7F0FD0020FFF7EDFD0020FFF7EAFDBF
:105110008020FFF7E7FDFC20FFF7E4FD8020FFF78C
:10512000E1FD0020FFF7DEFD8020FFF7DBFDFC2026
:10513000FFF7D8FDF820FFF7D5FD0020FFF7D2FDDF
:105140006020FFF7CFFDBC20FFF7CCFD6020FFF70C
:10515000C9FD0020FFF7C6FD6020FFF7C3FDBC209E
:10516000FFF7C0FDB820FFF7BDFD0020FFF7BAFD37
:105170000027BDB2002429462046DFF747F8DFF7B5
:1051800073F8FFF743FE0646601C294680B2DFF73E
:105190003DF8DFF769F8FFF739FE40EA0613D8B2A9
:1051A000FFF7A0FDA11C8CB220462946DFF72EF8A0
:1051B000DFF75AF8FFF72AFE621C2946064690B22E
:1051C000DFF724F8DFF750F8FFF720FE023440EA5B
:1051D0000610C0B2A4B2FFF785FDB4F5C87FCAD1EE
:1051E0000137F02FC5D1BDE8F840FFF7ABBD00BFD8
:1051F000CF81020847F29823C2F200031880188872
:1052000082B2002AFBD170472DE9F04F40F66A7850
:10521000054608FB00F0C71C30EA200028BF3846CE
:105220004AF2FF1EC0F24A4E8410BEFBF4F44FF463
:10523000224CC0F24A4C661C9CFBF6F696FBF5F736
:1052400098FBF7F089B006FB00F720200691014695
:1052500004920593DEF7FAFF07200021DEF7F6FF40
:1052600008202146DEF7F2FF00208021DEF7EEFF66
:1052700040F2444297FBF5F8C4F202025368012B56
:10528000FCD140F24442C4F2020251680129FCD030
:1052900006200121DEF7DAFF0320DEF7DBFF00281E
:1052A000FAD09624013CDEF7C5FFDEF7C3FF013CD0
:1052B000F8D1284602F0C0FC40F6DB71C4F2C90107
:1052C00002F00EFD0546304602F0B6FC01462846C7
:1052D00002F0BAFD0025B8F1000F03906FF0FE0355
:1052E0002E4640F3AF80049808F1FF32071C18BF28
:1052F0000127059E02F0010BDEF79CFF002E18BF70
:1053000047F00107C0B200252E460028ACBF8246F8
:105310004FF0000AFF28B4BF81464FF0FF09002F6D
:1053200040F0CE800124444500F08A80BBF1000F9C
:105330000ED0DEF77FFFC0B28245B8BF82468145FE
:10534000A8BF8146002F40F0E7800134444577D064
:10535000DEF770FF5FFA80FC6046E245B8BFE246C8
:10536000E145A8BFE146002F2DD002F065FC834641
:10537000204602F061FC039902F0B2FC019000F0BB
:1053800087FD01460198029100F0B8FD00210190CF
:1053900002F0A6FC029A0146104602F097FB014675
:1053A000584602F09DFC0146304602F091FB019BFD
:1053B000064603F10041584602F092FC0146284699
:1053C00002F086FB0546DEF735FFC0B28245B8BF66
:1053D00082468145A8BF81460134002FB5D002F036
:1053E0002BFC8346204602F027FC039902F078FC50
:1053F000019000F04DFD019B01461846029100F01E
:105400007DFD0021019002F06BFC0146029802F044
:105410005DFB0146584602F063FC0146304602F04F
:1054200057FB019A064602F10041584602F058FC2B
:105430000146284602F04CFB01344445054687D11D
:10544000C9EB0A03069F08EBD8783B604FEA680077
:1054500002F0F2FB07463946304602F0F5FC3946C9
:105460000446284602F0F0FC21460546204602F09C
:1054700037FC29460646284602F032FC01463046F3
:1054800002F026FB00F078FD049B06463BB140F29B
:10549000F341C3F6B57102F0D7FC049A1060059988
:1054A00059B130464FF0804102F0D6FD00285AD164
:1054B00000230598C7F6C073036009B0BDE8F08FFC
:1054C00002F0BAFB0790204602F0B6FB039902F007
:1054D00007FC044600F0DCFC0646204600F00EFD0A
:1054E0002946044602F0FCFB0146304602F0EEFA83
:1054F0000146079802F0F4FB0146284602F0E8FA5C
:1055000004F100410646079802F0EAFB01462846EE
:1055100002F0DEFA054605E702F08EFB83462046E0
:1055200002F08AFB039902F0DBFB029000F0B0FC72
:10553000029B01461846019100F0E0FC0021029018
:1055400002F0CEFB0146019802F0C0FA014658462F
:1055500002F0C6FB0146304602F0BAFA029A06464D
:1055600002F1004161E705F10041204600F002FD33
:105570000021C4F2343102F0B3FB01F0EDFF06A3C9
:10558000D3E9002302F066F902F04CFA059A1060A4
:1055900093E700BFAFF30080182D4454FB2109406E
:1055A00010B5002182B004460A20DEF74FFE02202B
:1055B000FFF720FE00222046134601A9FFF724FE34
:1055C000019B0020C72B77DD01210A20DEF73EFE7C
:1055D0000220FFF70FFE0022204601A91346FFF725
:1055E00013FE01990120C72966DD02210A20DEF79A
:1055F0002DFE0220FFF7FEFD00222046134601A9E2
:10560000FFF702FE019A0220C72A55DD03210A2076
:10561000DEF71CFE0220FFF7EDFD002220461346B8
:1056200001A9FFF7F1FD019B0320C72B44DD0421F5
:105630000A20DEF70BFE0220FFF7DCFD00222046E9
:1056400001A91346FFF7E0FD01990420C72933DDC6
:1056500005210A20DEF7FAFD0220FFF7CBFD00222C
:105660002046134601A9FFF7CFFD019A0520C72A5E
:1056700022DD06210A20DEF7E9FD0220FFF7BAFD50
:1056800000222046134601A9FFF7BEFD019B06201C
:10569000C72B11DD07210A20DEF7D8FD0220FFF716
:1056A000A9FD0022204601A91346FFF7ADFD019890
:1056B000C728CCBF0820072002B010BD70B50D462A
:1056C00082B02B46694601AA0646FFF79DFD009B66
:1056D000143BD22B9CBF43F20004C2F200040DD94C
:1056E0003046FFF75DFF43F20004C2F20004206081
:1056F0006946304601AA2B46FFF786FD0720DEF7F4
:10570000A9FD226802EB820100EB8100006902F032
:1057100093FA019902F0E4FA4FF41051C4F67411AF
:1057200002F092FB02B070BD2DE9F0410446104634
:10573000884602F081FA40F6DB71C4F2C90102F03A
:10574000CFFA0546404602F077FA0146284602F0B5
:105750007BFBB8F1000F074640F381804FEA480811
:105760000025002618F0020F284651D14FF4604161
:105770002846C4F2FF4102F0B3FA4FF46041C4F28C
:10578000FF4102F0A5F902F097FC39462080284637
:1057900002F09EF940F6DB71C4F2C901054602F041
:1057A0005BFC38B140F6DB712846C4F2C90102F057
:1057B0008DF90546284600F0A1FB022628E000F0FE
:1057C0009DFB4FF46041C4F2FF4102F089FA4FF4AF
:1057D0006041C4F2FF4102F07BF902F06DFC3946F2
:1057E000A053284602F074F940F6DB71C4F2C901F7
:1057F000054602F031FC40F6DB71C4F2C90118B174
:10580000284602F063F90546284600F077FB023689
:105810004FF46041C4F2FF4102F062FA4FF460417C
:10582000C4F2FF4102F054F902F046FC3946A0539D
:10583000284602F04DF940F6DB71C4F2C901054675
:1058400002F00AFC40F6DB710236C4F2C90118B15D
:10585000284602F03BF9054646452846AFD1BDE84B
:10586000F08100BF2DE9F0414FF4FA5404FB00F839
:105870004DF6836708F1FF35C4F21B37A7FB05130C
:105880009A0C01324AF2FF1CB8FBF2F1C0F24A4C0A
:105890004FF6FF7EBCFBF1F8F045A8BFF0464FF491
:1058A000224608F10104C0F24A4696FBF4F702FBD7
:1058B00007F707EB5005B5FBF0F54FF4A05C43F29A
:1058C000CC36C4F2000CB5F5FA5FA8BF4FF4FA5518
:1058D000C2F200064FF0000340F24444ACF8283016
:1058E000C4F2020430462946FFF71EFF23680F204A
:1058F00023F0010222602946DEF7A8FC0E20314683
:10590000DEF7A4FC21680D2041F00103236041462D
:10591000DEF79CFC07EB5500B0FBF5F0BDE8F0812D
:1059200010B54AF2FF14C0F24A44B4FBF0F4621C12
:1059300012F0010F08BF144610200021DEF786FC8C
:105940001120611EDEF782FC12206108DEF77EFC6A
:105950004FF422416308C0F24A415818B0FBF4F0FA
:1059600010BD00BF48F2F06043F20001C0F6020033
:10597000C2F20001884270B426D043F20414C2F28D
:105980000004A14220D2024652F8046B0B46CD43DC
:1059900043F8046B6519A342C5F3800514D23DB1E9
:1059A000156800F108021D6001F10803A3420BD243
:1059B000114651F8045B1846526840F8045B5A607F
:1059C000031D0A1DA342F3D343F2041247F2B4208D
:1059D000C2F20002C2F20000824216D20021134637
:1059E000D44343F8041B04198342C4F380040CD24B
:1059F00024B1196002F10803834206D21A4642F824
:105A0000041B5960131D8342F8D370BC704700BF5C
:105A1000DFF828D044F2000369464FF46D42C0F627
:105A20000203CEF20002C2F200018D469360FFF73E
:105A300099FFDEF71BFCFEF77BFBFEE700C00020B2
:105A4000F0B547F24C24C2F200040A2883B027685C
:105A500007D03F2F05D0E11901370871276003B047
:105A6000F0BD0026E71943F20405C2F200053E71BD
:105A7000064F334629880A204FF6FF720097DEF75B
:105A8000E3FB2B6826600E3B2B60E8E7507200209A
:105A900010B50446007828B1FFF7D2FF14F8010FC3
:105AA0000028F9D110BD00BF10B50446C078000928
:105AB000092839DD3730FFF7C3FFE17801F00F0027
:105AC000092839DD3730FFF7BBFFA2781009092814
:105AD00039DD3730FFF7B4FFA37803F00F00092852
:105AE00039DD3730FFF7ACFF60780009092839DD70
:105AF0003730FFF7A5FF617801F00F00092839DD85
:105B00003730FFF79DFF22781009092839DC303043
:105B1000FFF796FF237803F00F00092839DC3030B7
:105B2000BDE81040FFF78CBF3030FFF789FFE17808
:105B300001F00F000928C5DC3030FFF781FFA278A3
:105B400010090928C5DC3030FFF77AFFA37803F08D
:105B50000F000928C5DC3030FFF772FF60780009BC
:105B60000928C5DC3030FFF76BFF617801F00F00CA
:105B70000928C5DC3030FFF763FF227810090928B7
:105B8000C5DD3730FFF75CFF237803F00F000928ED
:105B9000C5DD3730C4E700BF704700BF002038B50F
:105BA0000146DEF733FB5E484BF68031DEF73CFB07
:105BB0005B484BF68031DEF737FB00210320DEF730
:105BC00045FB48F25020C0F60200FFF761FF47F2A4
:105BD0004C2448F28020C2F20004C0F60200FFF715
:105BE00057FF04F14400FFF75FFF48F28820C0F63A
:105BF0000200FFF74DFF606C00251830FFF754FFDF
:105C000048F29020C0F60200FFF742FF606C1430AB
:105C1000FFF74AFF48F29820C0F60200FFF738FF6E
:105C2000606CFFF741FF48F2A420C0F60200FFF7C6
:105C30002FFF606C0430FFF737FF48F2AC20C0F64E
:105C40000200FFF725FF606C0830FFF72DFF48F2D8
:105C5000B820C0F60200FFF71BFF606C0C30FFF7A6
:105C600023FF48F2C020C0F60200FFF711FF606C6E
:105C70001030FFF719FF48F2C820C0F60200FFF706
:105C800007FF4EF62C50CEF20000FFF70DFF48F252
:105C9000D420C0F60200FFF7FBFE4EF62850CEF2ED
:105CA0000000FFF701FF48F2E020C0F60200FFF716
:105CB000EFFE08E048F27C20C0F602000135FFF755
:105CC000E7FE202D25D0606C00EB8500FFF7ECFE91
:105CD00005F00302032A48F27C20C0F6020004BF4C
:105CE00048F2EC20C0F60200FFF7D2FE616C0135ED
:105CF00001EB8500FFF7D8FE05F00303032BD9D194
:105D000048F2EC20C0F602000135FFF7C1FE202D5D
:105D1000D9D148F2EC20C0F60200FFF7B9FEFEE749
:105D20000830002047F24C23C2F20003EFF3088250
:105D30005A64FFF733FF00BFFEE700BFFEE700BF76
:105D4000FEE700BFDEF75CBADEF75CBA38B547F2B3
:105D50004C24C2F20004A16C13204A1C0021A2644E
:105D6000DEF774FAB4F84C0083B223B1B4F84C00F7
:105D7000431EA4F84C3094F84E2047F24C23C2F254
:105D80000003002A59D1142283F84E201D6D15B14D
:105D9000186D411E1965B4F854C047F24C231FFA20
:105DA0008CF5132DC2F200034DD9B3F8542047F2FD
:105DB0004C25143AA3F8542094F856E0C2F200059A
:105DC000BEF1310F4CD895F856104B1C85F8563063
:105DD00094F85C0047F24C23421C84F85C2094F851
:105DE0005C10C2F200030B290ED9002283F85C205C
:105DF00093F85DE0DEF1010C38BF4FF0000C01219B
:105E000083F85DC083F85E1094F85F0047F24C237E
:105E1000C2F2000320B193F85F20511E83F85F1097
:105E200094F8600047F24C23C2F2000320B193F8CB
:105E30006020511E83F8601038BD93F84E00411E5B
:105E400083F84E1038BD03200021DEF7FFF994F8E7
:105E500056E047F24C25BEF1310FC2F20005B2D92F
:105E600000220420012185F85620DEF7EFF9B5F86D
:105E700058104B1CA5F85830B5F85A2090B200289D
:105E8000A6D0B5F85A30581EA5F85A00A0E700BFB2
:105E900040F6D87320F00042C3F6497301469A4297
:105EA00000B583B015DDB2F1FF4F03DB01F00EFE4C
:105EB00003B000BD694600F05DF900F003020098F0
:105EC000012A10D0022A08D09AB9019900F056FB95
:105ED000EEE7002100F052FBEAE7019900F04EFBEB
:105EE00000F10040E4E7019900F03AFF00F10040C2
:105EF000DEE70122019900F033FFD9E740F6D873BD
:105F000020F00042C3F6497301469A4200B583B0BF
:105F100016DDB2F1FF4F03DB01F0D8FD03B000BD89
:105F2000694600F027F900F00300012815D0022887
:105F30000BD0B8B900980122019900F011FFEDE7EC
:105F40000021002200F00CFFE8E7009801220199EF
:105F500000F006FF00F10040E0E70098019900F032
:105F60000DFBDBE70098019900F008FB00F1004011
:105F7000D4E700BF00F052B870B58AB0064600F012
:105F8000A5FA43F20C04C2F2000494F90030013384
:105F9000054630D0304601F0D5F800282BD03046E9
:105FA000002102F03BF830B348F2F0233046C0F64F
:105FB00002030193012300930023089301F0CCFA1C
:105FC0002478CDE90401CDE90201BCB10020002113
:105FD00002460B4601F03EFC022CCDE9060111D130
:105FE00002F08AF821230360089B8BB9DDE90601E2
:105FF00001F018FD054628460AB070BD00220023B6
:10600000CDE90623684600F02BFF0028ECD1E7E736
:1060100002F072F8089B0360E8E700BFF8B520F0D3
:106020000044B4F1FF4F21F00046D4BF0027012700
:10603000B6F1FF4FC8BF47F001070346002F45D117
:10604000B1F17E5F4CD08F1707F0020747EAD07797
:106050004CB9022F3FD0032F03D140F6DB73CCF2B3
:1060600049031846F8BD36B3B6F1FF4F55D0B4F129
:10607000FF4F20D0A41BE4153C2CC4BF40F6DB70BE
:10608000C3F6C97030DD012F08BF00F10043E8D02E
:10609000022F33D00346002FE3D04BF62E51C3F22C
:1060A000BB3101F015FD40F6DB71C4F2490101F08E
:1060B0000DFD0346D5E7002840F6DB73B8BFCBF6ED
:1060C000C973CEDBC3F6C9731846F8BD01F000FDF5
:1060D00003461846F8BD40F6DB73C4F24903C0E737
:1060E000BDE8F84000F0BEBE14F13C0FACBF002488
:1060F000012414EAD1741DD00020C4E74BF62E51C0
:10610000C3F2BB3101F0E4FC014640F6DB70C4F29F
:10611000490001F0DBFC0346A3E7B4F1FF4F10D0C8
:10612000022FD8D0032F98D00023012F99D14FF000
:10613000004396E701F088FE00F0B2FF00F092FE07
:10614000A1E7022F04BF4CF6E433C4F2160388D053
:10615000032F04BF4CF6E433CCF2160381D0012F99
:1061600040F6DB7318BFC3F649737FF47AAFCBF602
:10617000497376E740F6D8732DE9F04FC3F64973BB
:1061800020F0004B89B09B4505460C4640F38C80BF
:106190004CF6E333C4F216039B4526DC00284FF48B
:1061A0007861C3F6C97140F3538101F08FFC4FF45D
:1061B0007D632BF00F0BC3F6C9739B45054600F0BA
:1061C000828044F243410126C3F2357101F07EFC26
:1061D00001462060284601F079FC44F24341C3F2B5
:1061E000357101F073FC606062E04FF47863C4F2D3
:1061F00049339B4540F38280BBF1FF4F5CDA4FEAA5
:10620000EB59A9F186094FEAC953C3EB0B0B58466A
:1062100001F02CFF01F010FD03460146584605939E
:1062200001F054FC4FF0874101F05AFD064601F0A1
:106230001DFF01F001FD014607463046069701F0BB
:1062400045FC4FF0874101F04BFD002103260790EC
:1062500001F0DAFE88B10326384600210DF1180856
:10626000013E01F0D1FE40B158F8047D0021013E0D
:10627000384601F0C9FE0028F6D13346924E05A8F3
:1062800021464A4601960226009600F053FA002D58
:1062900006460DDA22684642636802F10042226037
:1062A00003F10043636003E00026002308604B60B5
:1062B000304609B0BDE8F08F0146002601F006FC2B
:1062C00060602060F4E74FF488410126C3F2357125
:1062D00001F0FCFB4AF20831C2F68561054601F087
:1062E000F5FB01462060284601F0F0FB4AF2083138
:1062F000C2F6856101F0EAFB6060D9E700F0D0FEEC
:106300004FF68411C3F62271074601F0E9FC4FF005
:106310007C5101F0DDFB01F0A9FE064601F08CFC8A
:106320004FF47861C3F6C971824601F0D9FC014689
:10633000384601F0CBFB44F24341C3F2357180464D
:10634000504601F0CDFC1F2E8146404621DC48F22C
:10635000F823711EC0F602032BF0FF0253F8213020
:106360009A4216D0494601F0B1FB074620603946F3
:10637000404601F0ABFB494601F0A8FB002D6060F0
:1063800096DA07F1004700F100402760764260602E
:106390008EE749464FEAEB5B01F098FBC0F3C75329
:1063A0000746C3EB0B032060082BE0DD4FF4884168
:1063B0005046C3F2357101F093FC0746404639461A
:1063C00001F084FB03904046039901F07FFB3946BE
:1063D00001F07CFB4AF20831C2F68561074650465F
:1063E00001F07EFC394601F071FB81460398494675
:1063F00001F06CFBC0F3C7530746C3EB0B0B2060E7
:10640000BBF1190FD8BFDDF80C80B0DD4FF423418C
:106410005046C2F6856101F063FC07460398394691
:1064200001F054FB80460398414601F04FFB39468A
:1064300001F04CFB43F23211C2F28D410746504647
:1064400001F04EFC394601F041FB8146404689E7A8
:1064500001F03EFB4FF47D632BF00F0BC3F6C973C5
:106460009B45054614D044F243414FF0FF36C3F23A
:10647000357101F02DFB01462060284601F026FB16
:1064800044F24341C3F2357101F022FB60600FE733
:106490004FF488414FF0FF36C3F2357101F018FB1D
:1064A0004AF20831C2F68561054601F011FB01464A
:1064B0002060284601F00AFB4AF20831C2F68561E5
:1064C00001F006FB6060F3E67883020820F00042EA
:1064D0000346B2F1FF4F70B5044639D2002A35D0D9
:1064E00000283FDBC115B2F5000F09D210F40002FD
:1064F00040D15B0001321802FBD5C2F101028918BC
:1065000023F07F43A1F17F0223F40003D10743F47A
:10651000000348BF5B000026541019215B0035467C
:106520004FF08072A8189842DEBFC0EB03038518B5
:10653000B61852085B000139F4D113B106F001031B
:106540009E197610E40506F17C56A419204670BD0C
:10655000014601F0C5FB0146204601F0B9FA0446A8
:10656000204670BD014601F0B1FA014601F06CFC15
:106570000446EBE701228918C2E700BF2DE9F84382
:1065800020F00046B6F1485F05460F465BDA01F0A1
:106590006DFD002800F0CA802946284601F0A0FBC6
:1065A0004DF24E71CAF64751044601F099FB47F28D
:1065B000F641C3F20F1101F08BFA214601F090FB76
:1065C0004FF27C21C3F2934101F080FA214601F0A1
:1065D00087FB40F60151C3F2D07101F079FA2146F0
:1065E00001F07EFB40F66131C3F6B62101F06EFA90
:1065F000214601F075FB4AF6AB21C3F62A5101F0A2
:1066000067FA214601F06CFB804620464FF07C5132
:1066100001F066FB41460646204601F061FB394623
:106620000446284601F05CFB0146204601F04EFA84
:106630000146304601F04AFA01464FF07E5001F023
:1066400045FABDE8F883014601F04AFB4DF24E7170
:10665000CAF64751044601F043FB47F2F641C3F244
:106660000F1101F035FA214601F03AFB4FF27C217F
:10667000C3F2934101F02AFA214601F031FB40F6C2
:106680000151C3F2D07101F023FA214601F028FB39
:1066900040F66131C3F6B62101F018FA214601F047
:1066A0001FFB4AF6AB21C3F62A5101F011FA21462D
:1066B00001F016FB49F69913C3F699639E42804692
:1066C000A3DD0023C3F648739E4227DC06F17F4614
:1066D0004FF07E50314601F0F9F9814620464FF0E7
:1066E0007C5101F0FDFA314601F0F0F941460646D1
:1066F000204601F0F5FA39460446284601F0F0FA42
:106700000146204601F0E2F90146304601F0DEF98B
:106710000146484601F0DAF9BDE8F8834FF0000978
:106720000026C3F63879C3F69066D7E74FF07E505F
:10673000BDE8F8832DE9F04F151DDDB0D41E58BF1C
:10674000254648F290640493013B0293ED10669B4A
:10675000C0F6020425EAE5750746099554F823407A
:10676000EB43089102EBC303029A079416190693B0
:1067700015D40136AD1A679B00240DF18008B600D0
:1067800003EB85090020002D03DB59F8040001F01C
:1067900053FA48F8040004340135B442F2D1079C9E
:1067A000002C25DB079A48ABDDF810A00DF58E799B
:1067B00003EB820B4FEA8A08029C0025002C11DBB8
:1067C00020A8002400EB8A0600253859043456F826
:1067D000041D01F085FA0146284601F079F9444587
:1067E0000546F2D149F8045FD9450AF1010AE3D11F
:1067F000079A0CABDDF81C80013A0093C2460A925E
:1068000003EB82040B944FEA8A025CACA318BAF142
:10681000000F019253F8504C22DD0DF590790BAE2C
:1068200009EB02054FF06E51204601F059FA01F0D4
:106830001DFC01F001FA4FF08741804601F050FA4B
:106840000146204601F042F901F010FC414646F8AD
:10685000040F55F8040D01F03BF94D450446E1D114
:106860000699204600F0ACFC4FF07851044601F048
:1068700037FA00F019FC4FF0824101F031FA01467D
:10688000204601F023F9044601F0F0FB064601F032
:10689000D3F90146204601F019F9069A002A054667
:1068A00040F306810AF1FF330CA8C2F10801C2F1DE
:1068B000070450F8232052FA01F0361810FA01F1BB
:1068C000521A0CA942FA04FB41F82320BBF1000F35
:1068D00030DD01360024BAF1000F17DD019C0CAB4E
:1068E0001919002407E022B10124C2F5807243F88F
:1068F000042C8B420AD053F8042B002CF3D0012433
:106900008B42C2F1FF0243F8042CF4D1069A002A0C
:106910000DDD012A00F0D580022A08D10AF1FF33EB
:106920000CA951F8232002F03F0241F82320BBF1CB
:10693000020F6ED02846002101F066FB002800F00F
:106940008180079A0AF1FF34A2420FDC019A0CA859
:106950008318079A00EB8200002253F8041D83423B
:1069600042EA0102F9D1002A40F0C3800A9C0CA837
:1069700050F82430002B40F0BA800B9A012352F8D3
:10698000041D01330029FAD053440AF10109994545
:1069900003933BDC099C029AA244679C02EB090327
:1069A00020AA04EB8A0B049C013B059202EB830AAC
:1069B0004FEA8408019B48AAD21801925BF8040FA1
:1069C000002501F039F9029A002A4AF8040F14DB75
:1069D000049B0025059A002409EB030602EB8606BA
:1069E0003859043456F8041D01F07AF90146284656
:1069F00001F06EF844450546F2D1039C09F1010906
:106A0000019BA14543F8045F0193D7DDDDF80CA09D
:106A1000F9E629464FF07E5001F058F80546002C63
:106A200088D006994FF07E5000F0CAFB01462846F8
:106A300001F04CF800210546284601F0E5FA00284F
:106A40007FF47FAF0296D0460AF1FF34002851D17F
:106A5000069B2846594200F0B3FB4FF0874104469D
:106A600001F0F0FA002800F071814FF06E512046DD
:106A700001F036F9069A0AF101080832069201F08F
:106A8000F5FA01F0D9F84FF08741054601F028F9F1
:106A90000146204601F01AF80CAC01F0E7FA0CAB05
:106AA00043F82A00284601F0E1FA44F8280034E0CF
:106AB00011D10AF1FF330CAA52F823304FEA232BED
:106AC00004E70AF1FF330CA850F8232002F07F02FC
:106AD00040F823202BE74FF07C514FF0000B01F0E2
:106AE000B1FA00283FF426AF4FF0020BF1E6012384
:106AF0004AE702960CA8069AA04650F82430083AB5
:106B0000069253B900EB8403A04653F8041D08F124
:106B1000FF38083A0029F8D006924FF07E500699C7
:106B200000F04EFBB8F1000F05464CDB08F1010206
:106B30000CAB48A8019296009C19861954F8040DD4
:106B400001F07AF8294601F0CBF84FF06E5146F883
:106B5000040D284601F0C4F8009A94420546EDD190
:106B600048ABCDF80C8003EB8809DFF8F0A1DDF825
:106B70001C800027B8F1000FC0F2DA80002FC0F2AD
:106B8000D78000240026254601E0BD420EDC59F8DE
:106B9000041001355AF80400043401F0A1F801464C
:106BA000304600F095FFA8450646EEDA5CAC019A47
:106BB00004EB87030137BA42A9F1040943F8A06C3A
:106BC000D8D1DDF80C80669C032C14D8DFE804F0E3
:106BD000986868190020BBF1000F59D0089B00F19C
:106BE0000040089C349A9860359B02F10042226074
:106BF00003F100436360029A02F007005DB0BDE854
:106C0000F08FB8F1000FC4BF34AD05EB8804E1DDAF
:106C100054F8049C54F804794846394600F058FF6B
:106C200006464846314600F051FF0146384600F01E
:106C30004FFFAC4226606060EAD1B8F1010FC9DDB8
:106C400008F1FF3405EB840454F80499A76848461A
:106C5000394600F03DFF06464846314600F036FF13
:106C60000146384600F034FFAC426660A060EBD1CC
:106C700008F1010804F10805002004EB880454F829
:106C8000041D00F025FFAC42F9D1BBF1000FA5D1E6
:106C9000089B089C9860349B2360359B6360AAE73F
:106CA0000020B8F1000F0BDB08F1010434AD002027
:106CB00005EB840454F8041D00F00AFFAC42F9D13E
:106CC00000F10043BBF1000F00D10346089C0146D0
:106CD0003498236000F0FAFEB8F1000F08DD34AC00
:106CE00004EB880854F8041F00F0F2FE4445F9D183
:106CF000BBF1000F01D000F10040089A50607AE724
:106D00000020B8F1000F0BDB08F1010434AD0020C6
:106D100005EB840454F8041D00F0DAFEAC42F9D10E
:106D2000BBF1000F01D000F10040089A106062E74B
:106D30005CAC019A04EB870301370026BA42A9F143
:106D4000040943F8A06C7FF415AF3AE7204601F040
:106D50008DF90CA941F82A00DFE600BF9C860208E5
:106D60002DE9F84320F00043B3F1485F04460D4697
:106D7000904603DA01F07AF9002859D021462046DE
:106D800000F0AEFF2146064600F0AAFF4CF6D311F4
:106D9000C2F62E710746304600F0A2FF42F634716B
:106DA000C3F2D72100F092FE314600F099FF4EF673
:106DB0001B71C3F2386100F08BFE314600F090FF8A
:106DC00040F60151C3F6501100F080FE314600F04C
:106DD00087FF48F68901C3F6084100F079FE814635
:106DE000B8F1000F27D028464FF07C5100F078FF13
:106DF00049468046384600F073FF0146404600F0A1
:106E000065FE314600F06CFF294600F05FFE4AF651
:106E1000AB21C3F62A610546384600F061FF014602
:106E2000284600F055FE0146204600F04FFE04467D
:106E30002046BDE8F8830146304600F051FF4AF68F
:106E4000AB21C3F62A6100F041FE394600F048FF4D
:106E50000146204600F03CFE04462046BDE8F8838B
:106E6000002070472DE9F04120F00045B5F1A14F19
:106E7000044606460EDBB5F1FF4F00F3A480002860
:106E800040F6DB74C8BFC3F6C97440F3D98020460E
:106E9000BDE8F0814FF6FF73C3F6DF639D4200F358
:106EA000A780B5F1445FC0F295804FF0FF372146CF
:106EB000204600F015FF0146804600F011FF46F61F
:106EC000D711C3F68541054600F00AFF4DF659215A
:106ED000C3F64B5100F0FCFD294600F001FF46F6D9
:106EE0003531C3F6885100F0F3FD294600F0F8FE75
:106EF00042F66E61C3F6BA5100F0EAFD294600F091
:106F0000EFFE44F62511C3F6126100F0E1FD2946BB
:106F100000F0E6FE4AF6AB21C3F6AA6100F0D8FD08
:106F2000414600F0DDFE4AF22121CBF615518046A4
:106F3000284600F0D5FE4FF26B11C3F66E5100F0FB
:106F4000C5FD294600F0CCFE48F29571C3F69D516F
:106F500000F0BCFD294600F0C3FE48F63861C3F6D8
:106F6000E35100F0B3FD294600F0BAFE4CF6CD41E6
:106F7000C3F64C6100F0AAFD294600F0B1FE7B1C6F
:106F8000014651D048F2C865404600F0A1FDC0F668
:106F90000205214600F0A4FE05EB8703196900F005
:106FA00095FD214600F092FD014655F8270000F0BE
:106FB0008DFD002EB8BF00F10044FFF668AF044617
:106FC0002046BDE8F081014600F082FD04462046DF
:106FD000BDE8F0814FF2CA21C7F2491100F078FDF7
:106FE0004FF07E5101F038F800283FF45EAF4EE7D5
:106FF00000F056F84FF6FF73C3F697739D424FF6B5
:10700000FF7304461FDCC3F62F739D423DDC01462F
:10701000002700F05DFD4FF07E5100F057FD4FF06E
:107020008041054620461FE0404600F051FD2146C4
:1070300000F056FE0146204600F048FD044626E7D3
:10704000CBF6C97423E7C4F21B039D4214DC4FF056
:107050007F51022700F03AFD4FF07F510546204650
:1070600000F03EFE4FF07E5100F032FD0146284612
:1070700000F0EAFE04461AE700202146CBF68070B5
:10708000032700F0E1FE044611E74FF07E5101278F
:1070900000F01CFD4FF07E5105462046E4E700BF9E
:1070A00020F00040704700BF2DE9F04120F000467D
:1070B00001460446F50D7F3D162D1ADC002D804655
:1070C00020DB4FF6FF77C0F27F072F4107420DD03C
:1070D0004FF2CA21C7F2491100F0FAFC002100F07A
:1070E000BBFF10B3002C24DB28EA07010846BDE8EB
:1070F000F081B6F1FF4FF9D300F0EAFC01460846F3
:10710000BDE8F0814FF2CA21C7F2491100F0E0FC5E
:10711000002100F0A1FF40B10021002CE6DACBF6FF
:107120008071002E08BF2146E0E721460846BDE8F1
:10713000F0814FF4000353FA05F504EB050828EA43
:107140000701D3E7D0F1010338BF0023B0F1004FAE
:1071500008BF43F001030BB102207047A0F5000304
:1071600000F1FF42B3F1FE4F2CBF00230123B2F127
:10717000FE4F38BF43F001030BB1042070474FF6B8
:10718000FE73411EC0F27F0300F10042013A9942B2
:107190008CBF002101219A428CBF0B4641F00103B4
:1071A0000BB10320704710F5000F14BF002301231B
:1071B000B0F1FF4F14BF184643F00100704700BF05
:1071C00010B50C4630F000410346024627D0B1F11D
:1071D000FF4F26D2B1F5000F29D3C90D0919FE2999
:1071E000C8BF194633DC0029C4BF22F0FF4242EA7F
:1071F000C15314DC11F1160F37DA4CF25032194634
:10720000944224DC44F26020C0F6A25000F03AF828
:1072100044F26021C0F6A25100F062FD0346184618
:1072200010BD014600F054FC0346184610BD4FF057
:10723000984100F055FD43F6B042CFF6FF729442FC
:107240000346E5DBC0F3C75102461939C6E74FF2E2
:10725000CA20C7F2491000F015F84FF2CA21C7F250
:10726000491100F03DFD0346D9E701F1190022F074
:10727000FF424FF04C5142EAC05000F031FD03464E
:10728000CDE700BF01F0004120F000400843704707
:1072900081F0004102E000BF83F0004330B54FEAC7
:1072A00041044FEA430594EA050F08BF90EA020F34
:1072B0001FBF54EA000C55EA020C7FEA645C7FEAC7
:1072C000655C00F0E2804FEA5454D4EB5555B8BFEA
:1072D0006D420CDD2C4480EA020281EA030382EA5B
:1072E000000083EA010180EA020281EA0303362DED
:1072F00088BF30BD11F0004F4FEA01314FF4801CC0
:107300004CEA113102D0404261EB410113F0004FD1
:107310004FEA03334CEA133302D0524263EB430388
:1073200094EA050F00F0A780A4F10104D5F1200E26
:107330000DDB02FA0EFC22FA05F2801841F1000181
:1073400003FA0EF2801843FA05F359410EE0A5F155
:1073500020050EF1200E012A03FA0EFC28BF4CF086
:10736000020C43FA05F3C01851EBE37101F000453C
:1073700007D54FF0000EDCF1000C7EEB00006EEB49
:107380000101B1F5801F1BD3B1F5001F0CD34908D3
:107390005FEA30004FEA3C0C04F101044FEA44522A
:1073A00012F5800F80F09A80BCF1004F08BF5FEAB1
:1073B000500C50F1000041EB045141EA050130BD91
:1073C0005FEA4C0C404141EB010111F4801FA4F134
:1073D0000104E9D191F0000F04BF01460020B1FA89
:1073E00081F308BF2033A3F10B03B3F120020CDAC1
:1073F0000C3208DD02F1140CC2F10C0201FA0CF09F
:1074000021FA02F10CE002F11402D8BFC2F1200C03
:1074100001FA02F120FA0CFCDCBF41EA0C019040B9
:10742000E41AA2BF01EB0451294330BD6FEA040402
:107430001F3C1CDA0C340EDC04F11404C4F12002ED
:1074400020FA04F001FA02F340EA030021FA04F3FF
:1074500045EA030130BDC4F10C04C4F1200220FA56
:1074600002F001FA04F340EA0300294630BD21FA94
:1074700004F0294630BD94F0000F83F4801306BF5A
:1074800081F480110134013D4EE77FEA645C18BF4E
:107490007FEA655C29D094EA050F08BF90EA020FE5
:1074A00005D054EA000C04BF1946104630BD91EADD
:1074B000030F1EBF0021002030BD5FEA545C05D1E0
:1074C0004000494128BF41F0004130BD14F580041F
:1074D0003CBF01F5801130BD01F0004545F0FE4193
:1074E00041F470014FF0000030BD7FEA645C1ABFC8
:1074F000194610467FEA655C1CBF0B46024650EAFF
:10750000013406BF52EA033591EA030F41F400212A
:1075100030BD00BF90F0000F04BF0021704730B5B0
:107520004FF4806404F132044FF000054FF0000185
:1075300050E700BF90F0000F04BF0021704730B546
:107540004FF4806404F1320410F0004548BF40421B
:107550004FF000013EE700BF42004FEAE2014FEA70
:1075600031014FEA02701FBF12F07F4393F07F4F4B
:1075700081F06051704792F0000F14BF93F07F4F7D
:10758000704730B54FF4607401F0004521F00041C0
:1075900020E700BF50EA010208BF704730B54FF046
:1075A00000050AE050EA010208BF704730B511F04B
:1075B000004502D5404261EB41014FF4806404F183
:1075C00032045FEA915C3FF4DCAE4FF003025FEA05
:1075D000DC0C18BF03325FEADC0C18BF033202EB8D
:1075E000DC02C2F1200300FA03FC20FA02F001FAE7
:1075F00003FE40EA0E0021FA02F11444C1E600BF86
:1076000070B54FF0FF0C4CF4E06C1CEA11541DBF38
:107610001CEA135594EA0C0F95EA0C0F00F0DEF803
:107620002C4481EA030621EA4C5123EA4C5350EAE8
:10763000013518BF52EA033541F4801143F4801339
:1076400038D0A0FB02CE4FF00005E1FB02E506F0CA
:107650000042E0FB03E54FF00006E1FB03569CF01F
:10766000000F18BF4EF0010EA4F1FF04B6F5007F25
:1076700064F5407404D25FEA4E0E6D4146EB060697
:1076800042EAC62141EA55514FEAC52040EA5E5020
:107690004FEACE2EB4F1FD0C88BFBCF5E06F1ED8CA
:1076A000BEF1004F08BF5FEA500E50F1000041EB01
:1076B000045170BD06F0004646EA010140EA0200AE
:1076C00081EA0301B4EB5C04C2BFD4EB0C0541EAD0
:1076D000045170BD41F480114FF0000E013C00F3E5
:1076E000AB8014F1360FDEBF002001F0004170BD09
:1076F000C4F10004203C35DA0C341BDC04F1140422
:10770000C4F1200500FA05F320FA04F001FA05F2AD
:1077100040EA020001F0004221F0004110EBD3707A
:1077200021FA04F642EB06015EEA430E08BF20EAA6
:10773000D37070BDC4F10C04C4F1200500FA04F349
:1077400020FA05F001FA04F240EA020001F00041DB
:1077500010EBD37041F100015EEA430E08BF20EA4E
:10776000D37070BDC4F1200500FA05F24EEA020E96
:1077700020FA04F301FA05F243EA020321FA04F0C5
:1077800001F0004121FA04F220EA020000EBD3707C
:107790005EEA430E08BF20EAD37070BD94F0000F7C
:1077A0000FD101F00046400041EB010111F4801FB0
:1077B00008BF013CF7D041EA060195F0000F18BF61
:1077C000704703F00046520043EB030313F4801F9D
:1077D00008BF013DF7D043EA0603704794EA0C0F57
:1077E0000CEA135518BF95EA0C0F0CD050EA41066D
:1077F00018BF52EA4306D1D181EA030101F00041EA
:107800004FF0000070BD50EA410606BF1046194611
:1078100052EA430619D094EA0C0F02D150EA01361D
:1078200013D195EA0C0F05D152EA03361CBF10465E
:1078300019460AD181EA030101F0004141F0FE41FD
:1078400041F470014FF0000070BD41F0FE4141F481
:10785000780170BD70B54FF0FF0C4CF4E06C1CEA81
:1078600011541DBF1CEA135594EA0C0F95EA0C0F36
:1078700000F0A7F8A4EB050481EA030E52EA0335F1
:107880004FEA013100F088804FEA03334FF0805512
:1078900045EA131343EA12634FEA022245EA11153F
:1078A00045EA10654FEA00260EF000419D4208BFF0
:1078B000964244F1FD0404F5407402D25B084FEA9D
:1078C0003202B61A65EB03055B084FEA32024FF449
:1078D00080104FF4002CB6EB020E75EB030E22BFA6
:1078E000B61A754640EA0C005B084FEA3202B6EB66
:1078F000020E75EB030E22BFB61A754640EA5C0015
:107900005B084FEA3202B6EB020E75EB030E22BFA4
:10791000B61A754640EA9C005B084FEA3202B6EBA5
:10792000020E75EB030E22BFB61A754640EADC0064
:1079300055EA060E18D04FEA051545EA16754FEAC6
:1079400006164FEAC30343EA52734FEAC2025FEAE4
:107950001C1CC0D111F4801F0BD141EA00014FF073
:1079600000004FF0004CB6E711F4801F04BF014344
:107970000020B4F1FD0C88BFBCF5E06F3FF6AFAE60
:10798000B5EB030C04BFB6EB020C5FEA500C50F1F0
:10799000000041EB045170BD0EF0004E4EEA113173
:1079A00014EB5C04C2BFD4EB0C0541EA045170BD7A
:1079B00041F480114FF0000E013C90E645EA060EBE
:1079C0008DE60CEA135594EA0C0F08BF95EA0C0FEC
:1079D0003FF43BAF94EA0C0F0AD150EA01347FF434
:1079E00034AF95EA0C0F7FF425AF104619462CE70B
:1079F00095EA0C0F06D152EA03353FF4FDAE10466E
:107A0000194622E750EA410618BF52EA43067FF4BE
:107A1000C5AE50EA41047FF40DAF52EA43057FF44E
:107A2000EBAE12E74FEA4102B2F1E04324BFB3F5F7
:107A3000001CDCF1FE5C0DD901F0004C4FEAC002E5
:107A40004CEA5070B2F1004F40EB830008BF20F0C9
:107A50000100704711F0804F21D113F13872BCBF83
:107A600001F00040704741F480114FEA5252C2F1D8
:107A70001802C2F1200C10FA0CF320FA02F018BF21
:107A800040F001004FEAC1234FEAD32303FA0CFC74
:107A900040EA0C0023FA02F34FEA4303CCE77FEA03
:107AA000625307D150EA01331EBF4FF0FE4040F44D
:107AB0004000704701F0004040F0FE4040F40000FC
:107AC000704700BF80F0004002E000BF81F000413D
:107AD00042001FBF5FEA410392EA030F7FEA226C74
:107AE0007FEA236C6AD04FEA1262D2EB1363C1BF04
:107AF000D218414048404140B8BF5B42192B88BF73
:107B0000704710F0004F40F4000020F07F4018BF95
:107B1000404211F0004F41F4000121F07F4118BFB5
:107B2000494292EA030F3FD0A2F1010241FA03FC5D
:107B300010EB0C00C3F1200301FA03F100F0004345
:107B400002D5494260EB4000B0F5000F13D3B0F10D
:107B5000807F06D340084FEA310102F10102FE2A7C
:107B600051D2B1F1004F40EBC25008BF20F00100EC
:107B700040EA03007047490040EB000010F4000F9A
:107B8000A2F10102EDD1B0FA80FCACF1080CB2EB2D
:107B90000C0200FA0CF0AABF00EBC250524218438C
:107BA000BCBFD0401843704792F0000F81F4000131
:107BB00006BF80F400000132013BB5E74FEA410304
:107BC0007FEA226C18BF7FEA236C21D092EA030F70
:107BD00004D092F0000F08BF0846704790EA010FEA
:107BE0001CBF0020704712F07F4F04D1400028BF17
:107BF00040F00040704712F100723CBF00F50000F9
:107C0000704700F0004343F0FE4040F4000070472E
:107C10007FEA226216BF08467FEA236301464202DA
:107C200006BF5FEA412390EA010F40F480007047ED
:107C30004FF0000304E000BF10F0004348BF404293
:107C40005FEA000C08BF704743F0964301464FF0CF
:107C500000001CE050EA010208BF70474FF000032B
:107C60000AE000BF50EA010208BF704711F000436C
:107C700002D5404261EB41015FEA010C02BF84463C
:107C80000146002043F0B64308BFA3F18053A3F59B
:107C90000003BCFA8CF2083AA3EBC25310DB01FAE2
:107CA00002FC634400FA02FCC2F12002BCF1004F66
:107CB00020FA02F243EB020008BF20F001007047F7
:107CC00002F1200201FA02FCC2F1200250EA4C004B
:107CD00021FA02F243EB020008BF20EADC70704791
:107CE0004FF0FF0C1CEAD0521EBF1CEAD15392EA9F
:107CF0000C0F93EA0C0F6FD01A4480EA010C40027B
:107D000018BF5FEA41211ED04FF0006343EA5010D4
:107D100043EA5111A0FB01310CF00040B1F5000F16
:107D20003EBF490041EAD3715B0040EA010062F1C5
:107D30007F02FD2A1DD8B3F1004F40EBC25008BFAF
:107D400020F00100704790F0000F0CF0004C08BFCD
:107D500049024CEA502040EA51207F3AC2BFD2F19A
:107D6000FF0340EAC250704740F400004FF00003A8
:107D7000013A5DDC12F1190FDCBF00F000407047E2
:107D8000C2F10002410021FA02F1C2F1200200FA20
:107D900002FC5FEA310040F1000053EA4C0308BFE7
:107DA00020EADC70704792F0000F00F0004C02BF38
:107DB000400010F4000F013AF9D040EA0C0093F0B3
:107DC000000F01F0004C02BF490011F4000F013B0D
:107DD000F9D041EA0C018FE70CEAD15392EA0C0F7B
:107DE00018BF93EA0C0F0AD030F0004C18BF31F0E6
:107DF000004CD8D180EA010000F00040704790F0BC
:107E0000000F17BF90F0004F084691F0000F91F05F
:107E1000004F14D092EA0C0F01D142020FD193EA25
:107E20000C0F03D14B0218BF084608D180EA0100AD
:107E300000F0004040F0FE4040F40000704740F089
:107E4000FE4040F4400070474FF0FF0C1CEAD05257
:107E50001EBF1CEAD15392EA0C0F93EA0C0F69D0B3
:107E6000A2EB030280EA010C49024FEA402037D01E
:107E70004FF0805343EA111143EA10130CF0004015
:107E80008B4238BF5B0042F17D024FF4000C8B4205
:107E900024BF5B1A40EA0C00B3EB510F24BFA3EBE5
:107EA000510340EA5C00B3EB910F24BFA3EB9103B5
:107EB00040EA9C00B3EBD10F24BFA3EBD10340EA0F
:107EC000DC001B0118BF5FEA1C1CE0D1FD2A3FF655
:107ED00050AF8B4240EBC25008BF20F0010070470A
:107EE0000CF0004C4CEA50207F32C2BFD2F1FF03AD
:107EF00040EAC250704740F400004FF00003013ADE
:107F000037E792F0000F00F0004C02BF400010F481
:107F1000000F013AF9D040EA0C0093F0000F01F095
:107F2000004C02BF490011F4000F013BF9D041EAB7
:107F30000C0195E70CEAD15392EA0C0F08D14202EA
:107F40007FF47DAF93EA0C0F7FF470AF084676E7BD
:107F500093EA0C0F04D14B023FF44CAF08466EE796
:107F600030F0004C18BF31F0004CCAD130F0004264
:107F70007FF45CAF31F000437FF43CAF5FE700BFBC
:107F80004FF0FF3C06E000BF4FF0010C02E000BFE5
:107F90004FF0010C4DF804CD4FEA40024FEA410387
:107FA0007FEA226C18BF7FEA236C11D001B052EA3D
:107FB000530C18BF90EA010F58BFB2EB030088BF03
:107FC000C81738BF6FEAE17018BF40F00100704772
:107FD0007FEA226C02D15FEA402C05D17FEA236C54
:107FE000E4D15FEA412CE1D05DF8040B704700BF9B
:107FF000844608466146FFE70FB5FFF7C9FF002832
:1080000048BF10F1000F0FBD4DF808EDFFF7F4FF6A
:108010000CBF012000205DF808FB00BF4DF808ED03
:10802000FFF7EAFF34BF012000205DF808FB00BF26
:108030004DF808EDFFF7E0FF94BF012000205DF848
:1080400008FB00BF4DF808EDFFF7D2FF94BF0120F9
:1080500000205DF808FB00BF4DF808EDFFF7C8FFF2
:1080600034BF012000205DF808FB00BF4FEA40024A
:10807000B2F1FE4F0FD34FF09E03B3EB12620DD956
:108080004FEA002343F0004310F0004F23FA02F0C0
:1080900018BF404270474FF00000704712F1610F67
:1080A00001D1420205D110F0004008BF6FF000403E
:1080B00070474FF00000704742000ED2B2F1FE4F01
:1080C0000BD34FF09E03B3EB126209D44FEA0023A7
:1080D00043F0004323FA02F070474FF0000070476E
:1080E00012F1610F01D1420202D14FF0FF3070470F
:1080F0004FF00000704700BF43F21003C2F20003CC
:108100001868704720F0030110F00300C0F1000070
:1081100051F8043B00F1040C4FEACC0C6FF0000264
:108120001CBF22FA0CF213434FF0010C4CEA0C2C4A
:108130004CEA0C4CA3EB0C0222EA030212EACC122A
:1081400004BF51F8043B0430F4D013F0FF0F1FBFFD
:10815000013013F47F4F013013F47F0F18BF01304B
:10816000704700BF4C4344207479706520697320C8
:1081700025303878200000004F6666696369616CBD
:1081800020666C6173682073697A653A20256420E3
:108190006B4220004661696C2061742025783A208A
:1081A000257820005465737420636F6D706C65745E
:1081B000653A20657874726120666C61736820612D
:1081C000742030782530387820776F726B732E00EA
:1081D000424DF6BB000000000000760000002800C1
:1081E000000090010000F000000001000400000009
:1081F000000080BB00007017000070170000100026
:10820000000000000000000020202020202020206E
:10821000202020202020202020202020202020205E
:10822000202020202020202020202020202020204E
:10823000202020202020202020202020202020203E
:10824000202020202020202020202020202020004E
:10825000202020202020202020202020202020201E
:1082600020202020484152444641554C5420202093
:10827000202020202020202020202020200000005E
:108280000A53503A20000000202050433A200000BA
:1082900020204C523A2000000A524547533A20729F
:1082A000302000002C207231200000000A20202005
:1082B00020202072322000002C2072332000000089
:1082C0002C207231322000000A534342204846538A
:1082D000523A20000A53434220434653523A200068
:1082E0000A535441434B2044554D503A0A00000074
:1082F0007371727466000000000FC93F000F49409F
:1083000000CB9640000FC9400053FB4000CB164104
:1083100000ED2F41000F49410031624100537B4184
:10832000003A8A4100CB9641005CA34100EDAF4189
:10833000007EBC41000FC94100A0D5410031E2419F
:1083400000C2EE410053FB4100F20342003A0A42F0
:108350000083104200CB164200141D42005C2342F1
:1083600000A5294200ED2F4200363642007E3C42F5
:1083700000C74242000F4942A2000000F90000007D
:10838000830000006E0000004E000000440000006A
:108390001500000029000000FC000000270000007C
:1083A00057000000D1000000F5000000340000007C
:1083B000DD000000C0000000DB00000062000000E3
:1083C00095000000990000003C0000004300000000
:1083D0009000000041000000FE000000510000007D
:1083E00063000000AB000000DE000000BB000000E6
:1083F000C500000061000000B7000000240000007C
:108400006E0000003A000000420000004D00000035
:10841000D2000000E000000006000000490000005B
:108420002E000000EA00000009000000D10000005A
:10843000920000001C000000FE0000001D00000073
:10844000EB0000001C000000B1000000290000004B
:10845000A70000003E000000E800000082000000CD
:1084600035000000F50000002E000000BB000000F9
:108470004400000084000000E90000009C000000AF
:108480007000000026000000B40000005F00000043
:108490007E00000041000000390000009100000053
:1084A000D6000000390000008300000053000000E7
:1084B00039000000F40000009C000000840000006F
:1084C0005F0000008B000000BD000000F90000000C
:1084D000280000003B0000001F000000F800000022
:1084E00097000000FF000000DE0000000500000013
:1084F000980000000F000000EF0000002F000000B7
:10850000110000008B0000005A0000000A0000006B
:108510006D0000001F0000006D000000360000002C
:108520007E000000CF00000027000000CB0000000C
:1085300009000000B70000004F00000046000000E6
:108540003F000000660000009E0000005F00000089
:10855000EA0000002D000000750000002700000068
:10856000BA000000C7000000EB000000E5000000BA
:10857000F10000007B0000003D000000070000004B
:1085800039000000F70000008A00000052000000DF
:1085900092000000EA0000006B000000FB000000F9
:1085A0005F000000B10000001F0000008D0000000F
:1085B0005D000000080000005600000003000000FD
:1085C0003000000046000000FC0000007B000000BE
:1085D0006B000000AB000000F0000000CF000000C6
:1085E000BC000000200000009A000000F400000021
:1085F000360000001D000000A9000000E30000009C
:1086000091000000610000005E000000E600000034
:108610001B00000008000000650000009900000039
:10862000850000005F00000014000000A0000000B2
:1086300068000000400000008D000000FF00000006
:10864000D8000000800000004D0000007300000012
:1086500027000000310000000600000006000000B6
:108660001500000056000000CA0000007300000062
:10867000A8000000C900000060000000E200000047
:108680007B000000C00000008C0000006B000000B8
:108690000400000007000000090000000000C93FBE
:1086A0000000F0390000DA370000A2330000842E09
:1086B0000000502B0000C2270000D0220000C41F81
:1086C0000000C61B000044173863ED3EDA0F493F37
:1086D0005E987B3FDA0FC93F6937AC31682122339E
:1086E000B40F14336821A23314300020430000007B
:1086F00004000000DC0000001F0014000100000066
:108700001430002000000000000000000000000005
:108710000000000000000000000000000000000059
:1087200000000000EC8602080000000000000000CD
:108730000000000000000000000000000000000039
:108740000000000000000000000000000000000029
:108750000000000000000000000000000000000019
:108760000000000000000000000000000000000009
:1087700000000000000000000000000000000000F9
:1087800000000000000000000000000000000000E9
:1087900000000000000000000000000000000000D9
:1087A00000000000000000000000000000000000C9
:1087B00000000000000000000000000000000000B9
:1087C00000000000000000000000000000000000A9
:1087D0000000000000000000000000000000000099
:1087E0000000000000000000000000000000000089
:0487F0000000000085
:020000040806EC
:1040000000000FF000000FF000000FF000000FF0B4
:1040100000000FF000000FF000000FF000000FF0A4
:1040200000000FF000000FF000000FF000000FF094
:1040300000000FF000000FF000000FF000000FF084
:0400000508025A1182
:00000001FF
